C51 COMPILER V9.51   EZI2C_1_INT                                                           01/04/2014 15:52:40 PAGE 1   


C51 COMPILER V9.51, COMPILATION OF MODULE EZI2C_1_INT
OBJECT MODULE PLACED IN .\DP8051\DP8051_Keil_951\Debug\EZI2C_1_INT.obj
COMPILER INVOKED BY: C:\Program Files (x86)\Cypress\PSoC Creator\3.0\PSoC Creator\import\keil\pk51\9.51\C51\BIN\c51.exe 
                    -.\Generated_Source\PSoC3\EZI2C_1_INT.c NOIV LARGE MODDP2 OMF2 VB(1) PR(.\DP8051\DP8051_Keil_951\Debug\EZI2C_1_INT.lst) C
                    -D DB NOIP OT(2,SIZE) DF(DEBUG) INCDIR(.,.\Generated_Source\PSoC3) OJ(.\DP8051\DP8051_Keil_951\Debug\EZI2C_1_INT.obj)

line level    source

   1          /*******************************************************************************
   2          * File Name: EZI2C_1INT.c
   3          * Version 1.90
   4          *
   5          * Description:
   6          *  This file contains the code that operates during the interrupt service
   7          *  routine.  For this component, most of the runtime code is located in
   8          *  the ISR.
   9          *
  10          *******************************************************************************
  11          * Copyright 2008-2013, Cypress Semiconductor Corporation.  All rights reserved.
  12          * You may use this file only in accordance with the license, terms, conditions,
  13          * disclaimers, and limitations in the end user license agreement accompanying
  14          * the software package with which this file was provided.
  15          *******************************************************************************/
  16          
  17          #include "EZI2C_1_PVT.h"
  18          
  19          
  20          /*******************************************************************************
  21          * Function Name: EZI2C_1_ISR
  22          ********************************************************************************
  23          *
  24          * Summary:
  25          *  Handle Interrupt Service Routine.
  26          *
  27          * Parameters:
  28          *  EZI2C_1_dataPtrS1: global variable, which stores pointer to the
  29          *  data exposed to an I2C master for the first slave address.
  30          *
  31          *  EZI2C_1_rwOffsetS1: global variable, which stores offset for read
  32          *  and write operations, is set at each write sequence of the first slave
  33          *  address.
  34          *
  35          *  EZI2C_1_rwIndexS1: global variable, which stores pointer to the next
  36          *  value to be read or written for the first slave address.
  37          *
  38          * EZI2C_1_wrProtectS1: global variable, which stores offset where data
  39          *  is read only for the first slave address.
  40          *
  41          * EZI2C_1_bufSizeS1: global variable, which stores size of data array
  42          *  exposed to an I2C master for the first slave address.
  43          *
  44          *  EZI2C_1_dataPtrS2: global variable, which stores pointer to the
  45          *  data exposed to an I2C master for the second slave address.
  46          *
  47          *  EZI2C_1_rwOffsetS2: global variable, which stores offset for read
  48          *  and write operations, is set at each write sequence of the second slave
  49          *  device.
  50          *
  51          *  EZI2C_1_rwIndexS2: global variable, which stores pointer to the next
  52          *  value to be read or written for the second slave address.
  53          *
C51 COMPILER V9.51   EZI2C_1_INT                                                           01/04/2014 15:52:40 PAGE 2   

  54          * EZI2C_1_wrProtectS2: global variable, which stores offset where data
  55          *  is read only for the second slave address.
  56          *
  57          * EZI2C_1_bufSizeS2: global variable, which stores size of data array
  58          *  exposed to an I2C master for the second slave address.
  59          *
  60          * EZI2C_1_curState: global variable, which stores current state of an
  61          *  I2C state machine.
  62          *
  63          *  EZI2C_1_curStatus: global variable, which stores current status of
  64          *  the component.
  65          *
  66          * Return:
  67          *  EZI2C_1_rwOffsetS1: global variable, which stores offset for read
  68          *  and write operations, is set at each write sequence of the first slave
  69          *  address. Is reset if received slave address matches first slave address
  70          *  and next operation will be read.
  71          *
  72          *  EZI2C_1_rwIndexS1: global variable, which stores pointer to the next
  73          *  value to be read or written for the first slave address. Is set to
  74          *  EZI2C_1_rwOffsetS1 and than incremented if received slave address
  75          *  matches first slave address and next operation will be read.
  76          *
  77          *  EZI2C_1_rwOffsetS2: global variable, which stores offset for read
  78          *  and write operations, is set at each write sequence of the second slave
  79          *  address. This variable is changes if new sub-address is passed to slave.
  80          *
  81          *  EZI2C_1_rwIndexS2: global variable, which stores pointer to the next
  82          *  value to be read or written for the second slave address. This variable is 
  83          *  changes if new sub-address is passed to slave.
  84          *
  85          *******************************************************************************/
  86          CY_ISR(EZI2C_1_ISR)
  87          {
  88   1          /* Making these static so not wasting time allocating
  89   1          *  on the stack each time and no one else can see them 
  90   1          */
  91   1          static uint8  tmp8;
  92   1          static uint8  tmpCsr;
  93   1      
  94   1          #if(EZI2C_1_SUBADDR_WIDTH == EZI2C_1_SUBADDR_16BIT)
                      static uint16 tmp16;
                  #endif /* (EZI2C_1_SUBADDR_WIDTH == EZI2C_1_SUBADDR_16BIT) */
  97   1      
  98   1          /* Entry from interrupt
  99   1          *  In hardware address compare mode, we can assume we only get interrupted
 100   1          *  when a valid address is recognized. In software address compare mode,
 101   1          *  we have to check every address after a start condition.
 102   1          */
 103   1      
 104   1          /* Make a copy so that we can check for stop condition after we are done */
 105   1          tmpCsr = EZI2C_1_CSR_REG;
 106   1          
 107   1          /* Check to see if a Start/Address is detected - reset the state machine.
 108   1          *  Check for a Read/Write condition.
 109   1          */
 110   1          if(EZI2C_1_IS_BIT_SET(tmpCsr, EZI2C_1_CSR_ADDRESS)) 
 111   1          {
 112   2              #if(EZI2C_1_ADDRESSES == EZI2C_1_TWO_ADDRESSES)
              
                          /* Get slave address from data register */
                          tmp8 = ((EZI2C_1_DATA_REG >> EZI2C_1_ADDRESS_SHIFT) & EZI2C_1_SADDR_MASK);
C51 COMPILER V9.51   EZI2C_1_INT                                                           01/04/2014 15:52:40 PAGE 3   

              
                          if(tmp8 == EZI2C_1_addrS1)   /* Check for address 1  */
                          {
                              if(EZI2C_1_IS_BIT_SET(EZI2C_1_DATA_REG, EZI2C_1_READ_FLAG))
                              {  /* Prepare next read op, get data and place in register */
              
                                  /* Load first data byte  */
                                  EZI2C_1_DATA_REG = EZI2C_1_dataPtrS1[EZI2C_1_rwOffsetS1];
              
                                  /* ACK and transmit */
                                  EZI2C_1_CSR_REG = (EZI2C_1_CSR_ACK | EZI2C_1_CSR_TRANSMIT);
              
                                  /* Set index to offset */
                                  EZI2C_1_rwIndexS1 = EZI2C_1_rwOffsetS1;
              
                                  /* Advance to data location */
                                  EZI2C_1_rwIndexS1++;
              
                                  /* Set Read busy status */
                                  EZI2C_1_curStatus |= EZI2C_1_STATUS_RD1BUSY;
              
                                  /* Prepare for read transaction */
                                  EZI2C_1_curState = EZI2C_1_SM_DEV1_RD_DATA;
                              }
                              else  /* Start of a Write transaction, reset pointers, first byte is address */
                              {  /* Prepare next opeation to write offset */
              
                                  /* ACK and ready to receive sub address */
                                  EZI2C_1_CSR_REG = EZI2C_1_CSR_ACK;
              
                                  /* Set Write busy status */
                                  EZI2C_1_curStatus |= EZI2C_1_STATUS_WR1BUSY;
              
                                  /* Prepare for read transaction */
                                  EZI2C_1_curState = EZI2C_1_SM_DEV1_WR_ADDR;
              
                                  /* Stop Interrupt Enable */
                                  EZI2C_1_CFG_REG  |= EZI2C_1_CFG_STOP_IE;
              
                              }  /* Prepared for the next Write transaction */
                          }   /* Slave address #1 is processed */
                          else if(tmp8 == EZI2C_1_addrS2)   /* Check for address 2  */
                          {
                              if(EZI2C_1_IS_BIT_SET(EZI2C_1_DATA_REG, EZI2C_1_READ_FLAG))
                              {  /* Prepare next read op, get data and place in register */
              
                                  /* Load first data byte  */
                                  EZI2C_1_DATA_REG = EZI2C_1_dataPtrS2[EZI2C_1_rwOffsetS2];
              
                                  /* ACK and transmit */
                                  EZI2C_1_CSR_REG = (EZI2C_1_CSR_ACK | EZI2C_1_CSR_TRANSMIT);
              
                                  /* Reset pointer to previous offset */
                                  EZI2C_1_rwIndexS2 = EZI2C_1_rwOffsetS2;
              
                                  /* Advance to data location */
                                  EZI2C_1_rwIndexS2++;
              
                                  /* Set read busy status */
                                  EZI2C_1_curStatus |= EZI2C_1_STATUS_RD2BUSY;
              
                                  /* Prepare for read transaction */
C51 COMPILER V9.51   EZI2C_1_INT                                                           01/04/2014 15:52:40 PAGE 4   

                                  EZI2C_1_curState = EZI2C_1_SM_DEV2_RD_DATA;
              
                              }  /* Prepared for the next Read transaction */
                              else  /* Start of a write trans, reset ptrs, 1st byte is addr */
                              {  /* Prepare next opeation to write offset */
              
                                  /* ACK and ready to receive addr */
                                  EZI2C_1_CSR_REG = EZI2C_1_CSR_ACK;
              
                                  /* Set Write busy status */
                                  EZI2C_1_curStatus |= EZI2C_1_STATUS_WR2BUSY;
              
                                  /* Prepare for read transaction */
                                  EZI2C_1_curState = EZI2C_1_SM_DEV2_WR_ADDR;
              
                                  /* Enable interrupt on Stop */
                                  EZI2C_1_CFG_REG  |= EZI2C_1_CFG_STOP_IE;
                              } /* Prepared for the next Write transaction */
                          }
                          else   /* No address match */
                          {   /* NAK address Match  */
                              EZI2C_1_CSR_REG = EZI2C_1_CSR_NAK;
                          }
                      #else /* One slave address - hardware address matching */
 202   2                  
 203   2                  if(EZI2C_1_IS_BIT_SET(EZI2C_1_DATA_REG, EZI2C_1_READ_FLAG))
 204   2                  {   /* Prepare next read op, get data and place in register */
 205   3      
 206   3                      /* Load first data byte  */
 207   3                      EZI2C_1_DATA_REG = EZI2C_1_dataPtrS1[EZI2C_1_rwOffsetS1];
 208   3      
 209   3                      /* ACK and transmit */
 210   3                      EZI2C_1_CSR_REG = (EZI2C_1_CSR_ACK | EZI2C_1_CSR_TRANSMIT);
 211   3      
 212   3                      /* Reset pointer to previous offset */
 213   3                      EZI2C_1_rwIndexS1 = EZI2C_1_rwOffsetS1;
 214   3      
 215   3                      /* Advance to data location */
 216   3                      EZI2C_1_rwIndexS1++;
 217   3      
 218   3                      /* Set read busy status */
 219   3                      EZI2C_1_curStatus |= EZI2C_1_STATUS_RD1BUSY;
 220   3      
 221   3                      /* Prepare for read transaction */
 222   3                      EZI2C_1_curState = EZI2C_1_SM_DEV1_RD_DATA;
 223   3                  }
 224   2                  else  /* Start of a write trans, reset ptrs, 1st byte is address */
 225   2                  {   /* Prepare next opeation to write offset */
 226   3      
 227   3                      /* ACK and ready to receive addr */
 228   3                      EZI2C_1_CSR_REG = EZI2C_1_CSR_ACK;
 229   3      
 230   3                      /* Set Write activity */
 231   3                      EZI2C_1_curStatus |= EZI2C_1_STATUS_WR1BUSY;
 232   3      
 233   3                      /* Prepare for read transaction */
 234   3                      EZI2C_1_curState = EZI2C_1_SM_DEV1_WR_ADDR;
 235   3      
 236   3                      /* Enable interrupt on stop */
 237   3                      EZI2C_1_CFG_REG |= EZI2C_1_CFG_STOP_IE;
 238   3                  }
 239   2              #endif  /* (EZI2C_1_ADDRESSES == EZI2C_1_TWO_ADDRESSES) */
C51 COMPILER V9.51   EZI2C_1_INT                                                           01/04/2014 15:52:40 PAGE 5   

 240   2          }
 241   1          else if(EZI2C_1_IS_BIT_SET(tmpCsr, EZI2C_1_CSR_BYTE_COMPLETE))
 242   1          {   /* Check for data transfer */
 243   2              
 244   2              /* Data transfer state machine */
 245   2              switch(EZI2C_1_curState)
 246   2              {
 247   3                  /* Address written from Master to Slave. */
 248   3                  case EZI2C_1_SM_DEV1_WR_ADDR:
 249   3      
 250   3                      /* If 8-bit interface, Advance to WR_Data, else to ADDR2 */
 251   3                      #if(EZI2C_1_SUBADDR_WIDTH == EZI2C_1_SUBADDR_8BIT)
 252   3                          
 253   3                          tmp8 = EZI2C_1_DATA_REG;
 254   3                          if(tmp8 < EZI2C_1_bufSizeS1)
 255   3                          {
 256   4                              /* ACK and ready to receive data */
 257   4                              EZI2C_1_CSR_REG = EZI2C_1_CSR_ACK;
 258   4      
 259   4                              /* Set offset to new value */
 260   4                              EZI2C_1_rwOffsetS1 = tmp8;
 261   4      
 262   4                              /* Reset index to offset value */
 263   4                              EZI2C_1_rwIndexS1 = tmp8;
 264   4      
 265   4                              /* Prepare for write transaction */
 266   4                              EZI2C_1_curState = EZI2C_1_SM_DEV1_WR_DATA;
 267   4                          }
 268   3                          else    /* Out of range, NAK data and don't set offset */
 269   3                          {
 270   4                              /* NAK the master */
 271   4                              EZI2C_1_CSR_REG = EZI2C_1_CSR_NAK;
 272   4                          }
 273   3      
 274   3                      #else   /* 16-bit */
              
                                  /* Save MSB of address */
                                  tmp16 = EZI2C_1_DATA_REG;
              
                                  /* ACK and ready to receive addr */
                                  EZI2C_1_CSR_REG = EZI2C_1_CSR_ACK;
              
                                  /* Prepare to get LSB of Addr */
                                  EZI2C_1_curState = EZI2C_1_SM_DEV1_WR_ADDR_LSB;
              
                              #endif  /* (EZI2C_1_SUBADDR_WIDTH == EZI2C_1_SUBADDR_8BIT) */
 286   3      
 287   3                  break;  /* case EZI2C_1_SM_DEV1_WR_ADDR */
 288   3      
 289   3                  #if(EZI2C_1_SUBADDR_WIDTH == EZI2C_1_SUBADDR_16BIT)
              
                              /* Only used with 16-bit interface */
                              case EZI2C_1_SM_DEV1_WR_ADDR_LSB:
              
                                  /* Create offset */
                                  tmp16 = (uint16) (tmp16 << EZI2C_1_ADDRESS_LSB_SHIFT) | EZI2C_1_DATA_REG;
              
                                  /* Check range */
                                  if(tmp16 < EZI2C_1_bufSizeS1)
                                  {
                                      /* ACK and ready to receive addr */
                                      EZI2C_1_CSR_REG = EZI2C_1_CSR_ACK;
C51 COMPILER V9.51   EZI2C_1_INT                                                           01/04/2014 15:52:40 PAGE 6   

              
                                      /* Set offset to new value */
                                      EZI2C_1_rwOffsetS1 = tmp16;
              
                                      /* Reset index to offset value */
                                      EZI2C_1_rwIndexS1 = tmp16;
              
                                      /* Prepare for write transaction */
                                      EZI2C_1_curState = EZI2C_1_SM_DEV1_WR_DATA;
                                  }
                                  else    /* Out of range, NAK data and don't set offset */
                                  {
                                      /* NAK the master */
                                      EZI2C_1_CSR_REG = EZI2C_1_CSR_NAK;
                                  }
                              break; /* case EZI2C_1_SM_DEV1_WR_ADDR_LSB */
              
                          #endif  /* (EZI2C_1_SUBADDR_WIDTH == EZI2C_1_SUBADDR_16BIT) */
 320   3      
 321   3      
 322   3                  /* Data written from Master to Slave. */
 323   3                  case EZI2C_1_SM_DEV1_WR_DATA:
 324   3                      
 325   3                      /* Check for valid range */
 326   3                      if(EZI2C_1_rwIndexS1 < EZI2C_1_wrProtectS1)
 327   3                      {
 328   4                          /* Get data, to ACK quickly */
 329   4                          tmp8 = EZI2C_1_DATA_REG;
 330   4      
 331   4                          /* ACK and ready to receive sub addr */
 332   4                          EZI2C_1_CSR_REG = EZI2C_1_CSR_ACK;
 333   4      
 334   4                          /* Write data to array */
 335   4                          EZI2C_1_dataPtrS1[EZI2C_1_rwIndexS1] = tmp8;
 336   4      
 337   4                          /* Increment pointer */
 338   4                          EZI2C_1_rwIndexS1++;
 339   4                      }
 340   3                      else
 341   3                      {
 342   4                          /* NAK cause beyond write area */
 343   4                          EZI2C_1_CSR_REG = EZI2C_1_CSR_NAK;
 344   4                      }
 345   3                  break;  /* EZI2C_1_SM_DEV1_WR_DATA */
 346   3      
 347   3      
 348   3                  /* Data read by Master from Slave */
 349   3                  case EZI2C_1_SM_DEV1_RD_DATA:
 350   3      
 351   3                      /* Check ACK/NAK */
 352   3                      if((tmpCsr & EZI2C_1_CSR_LRB) == EZI2C_1_CSR_LRB_ACK)
 353   3                      {
 354   4                          /* Check for valid range */
 355   4                          if(EZI2C_1_rwIndexS1 < EZI2C_1_bufSizeS1)
 356   4                          {
 357   5                              /* Get data from array */
 358   5                              EZI2C_1_DATA_REG = EZI2C_1_dataPtrS1[EZI2C_1_rwIndexS1];
 359   5      
 360   5                              /* Send Data */
 361   5                              EZI2C_1_CSR_REG = EZI2C_1_CSR_TRANSMIT;
 362   5      
 363   5                              /* Increment pointer */
C51 COMPILER V9.51   EZI2C_1_INT                                                           01/04/2014 15:52:40 PAGE 7   

 364   5                              EZI2C_1_rwIndexS1++;
 365   5                          }
 366   4                          else    /* No valid range */
 367   4                          {
 368   5                              /* Out of range send FFs */
 369   5                              EZI2C_1_DATA_REG = EZI2C_1_DUMMY_DATA;
 370   5      
 371   5                              /* Send Data */
 372   5                              EZI2C_1_CSR_REG = EZI2C_1_CSR_TRANSMIT;
 373   5                          }
 374   4                      }
 375   3                      else    /* Data was NAKed */
 376   3                      {
 377   4                          /* Send dummy data at the end of read transaction */
 378   4                          EZI2C_1_DATA_REG = EZI2C_1_DUMMY_DATA;
 379   4      
 380   4                          /* Clear transmit bit at the end of read transaction */
 381   4                          EZI2C_1_CSR_REG = EZI2C_1_CSR_NAK;
 382   4                          
 383   4                          /* Clear Busy Flag */
 384   4                          EZI2C_1_curStatus &= ((uint8) ~EZI2C_1_STATUS_BUSY);
 385   4      
 386   4                          /* Error or Stop, reset state */
 387   4                          EZI2C_1_curState = EZI2C_1_SM_IDLE;
 388   4      
 389   4                      }
 390   3                  break;  /* EZI2C_1_SM_DEV1_RD_DATA */
 391   3      
 392   3                  /* Second Device Address */
 393   3                  #if(EZI2C_1_ADDRESSES == EZI2C_1_TWO_ADDRESSES)
              
                              case EZI2C_1_SM_DEV2_WR_ADDR:
              
                                  /* If 8-bit interface, Advance to WR_Data, else to ADDR2 */
                                  #if(EZI2C_1_SUBADDR_WIDTH == EZI2C_1_SUBADDR_8BIT)
                                      
                                      tmp8 = EZI2C_1_DATA_REG;
                                      if(tmp8 < EZI2C_1_bufSizeS2)
                                      {
                                          /* ACK and ready to receive addr */
                                          EZI2C_1_CSR_REG = EZI2C_1_CSR_ACK;
              
                                          /* Set offset to new value */
                                          EZI2C_1_rwOffsetS2 = tmp8;
              
                                          /* Reset index to offset value */
                                          EZI2C_1_rwIndexS2 = tmp8;
              
                                          /* Prepare for write transaction */
                                          EZI2C_1_curState = EZI2C_1_SM_DEV2_WR_DATA;
                                      }
                                      else    /* Out of range, NAK data and don't set offset */
                                      {
                                          /* NAK the master */
                                          EZI2C_1_CSR_REG = EZI2C_1_CSR_NAK;
                                      }
                                  #else
                                      /* Save LSB of address */
                                      tmp16 = EZI2C_1_DATA_REG;
              
                                      /* ACK and ready to receive addr */
                                      EZI2C_1_CSR_REG = EZI2C_1_CSR_ACK;
C51 COMPILER V9.51   EZI2C_1_INT                                                           01/04/2014 15:52:40 PAGE 8   

              
                                      /* Prepare to get LSB of Addr */
                                      EZI2C_1_curState = EZI2C_1_SM_DEV2_WR_ADDR_LSB;
                                  #endif  /* (EZI2C_1_SUBADDR_WIDTH == EZI2C_1_SUBADDR_8BIT) */
              
                              break;  /* EZI2C_1_SM_DEV2_WR_ADDR */
              
                              #if(EZI2C_1_SUBADDR_WIDTH == EZI2C_1_SUBADDR_16BIT)
              
                                  /* Only used with 16-bit interface */
                                  case EZI2C_1_SM_DEV2_WR_ADDR_LSB:
                                      /* Create offset */
                                      tmp16 = (uint16) (tmp16 << 8u) | EZI2C_1_DATA_REG;
                                      if(tmp16 < EZI2C_1_bufSizeS2)
                                      {
                                          /* ACK and ready to receive addr */
                                          EZI2C_1_CSR_REG = EZI2C_1_CSR_ACK;
              
                                          /* Set offset to new value */
                                          EZI2C_1_rwOffsetS2 = tmp16;
              
                                          /* Reset index to offset value */
                                          EZI2C_1_rwIndexS2 = tmp16;
              
                                          /* Prepare for write transaction */
                                          EZI2C_1_curState = EZI2C_1_SM_DEV2_WR_DATA;
                                      }
                                      else    /* Out of range, NAK data and don't set offset */
                                      {
                                          /* NAK the master */
                                          EZI2C_1_CSR_REG = EZI2C_1_CSR_NAK;
                                      }
                                      break; /* EZI2C_1_SM_DEV2_WR_ADDR_LSB */
              
                              #endif   /* (EZI2C_1_SUBADDR_WIDTH == EZI2C_1_SUBADDR_16BIT) */
              
              
                              /* Data written from Master to Slave. */
                              case EZI2C_1_SM_DEV2_WR_DATA:
                                  
                                  /* Check for valid range */
                                  if(EZI2C_1_rwIndexS2 < EZI2C_1_wrProtectS2)
                                  {
                                      /* Get data, to ACK quickly */
                                      tmp8 = EZI2C_1_DATA_REG;
              
                                      /* ACK and ready to receive sub addr */
                                      EZI2C_1_CSR_REG = EZI2C_1_CSR_ACK;
              
                                      /* Write data to array */
                                      EZI2C_1_dataPtrS2[EZI2C_1_rwIndexS2] = tmp8;
              
                                      /* Inc pointer */
                                      EZI2C_1_rwIndexS2++;
                                  }
                                  else
                                  {
                                      /* NAK cause beyond write area */
                                      EZI2C_1_CSR_REG = EZI2C_1_CSR_NAK;
                                  }
                                  break;  /* EZI2C_1_SM_DEV2_WR_DATA */
              
C51 COMPILER V9.51   EZI2C_1_INT                                                           01/04/2014 15:52:40 PAGE 9   

                                  /* Data read by Master from Slave */
                                  case EZI2C_1_SM_DEV2_RD_DATA:
                                  
                                      if((tmpCsr & EZI2C_1_CSR_LRB) == EZI2C_1_CSR_LRB_ACK)
                                      {   /* ACKed */
                                          /* Check for valid range */
                                          if(EZI2C_1_rwIndexS2 < EZI2C_1_bufSizeS2)
                                          {   /* Check ACK/NAK */
                                              /* Get data from array */
                                              EZI2C_1_DATA_REG = EZI2C_1_dataPtrS2[EZI2C_1_rwIndexS2];
              
                                              /* Send Data */
                                              EZI2C_1_CSR_REG = EZI2C_1_CSR_TRANSMIT;
              
                                              /* Increment pointer */
                                              EZI2C_1_rwIndexS2++;    
                                          }
                                          else    /* Not valid range */
                                          {
                                              /* Out of range send FFs */
                                              EZI2C_1_DATA_REG = EZI2C_1_DUMMY_DATA;
              
                                              /* Send Data */
                                              EZI2C_1_CSR_REG = EZI2C_1_CSR_TRANSMIT;
                                          }
                                      }
                                      else    /* NAKed */
                                      {
                                          /* Out of range send FFs */
                                          EZI2C_1_DATA_REG = EZI2C_1_DUMMY_DATA;
              
                                          /* Send Data */
                                          EZI2C_1_CSR_REG = EZI2C_1_CSR_TRANSMIT;
              
                                          /* Clear busy status */
                                          EZI2C_1_curStatus &= ((uint8) ~EZI2C_1_STATUS_BUSY);
              
                                          /* Error or Stop, reset state */
                                          EZI2C_1_curState = EZI2C_1_SM_IDLE;
                                      }   /* End if ACK/NAK */
                                          
                                      break;  /* EZI2C_1_SM_DEV2_RD_DATA */
              
                          #endif  /* (EZI2C_1_ADDRESSES == EZI2C_1_TWO_ADDRESSES) */
 532   3      
 533   3                  default:
 534   3                      /* Invalid state, Reset */
 535   3                      EZI2C_1_curState = EZI2C_1_SM_IDLE;
 536   3      
 537   3                      /* Reset offsets and index */
 538   3                      EZI2C_1_rwOffsetS1 = 0u;
 539   3      
 540   3                      /* Clear index */
 541   3                      EZI2C_1_rwIndexS1 = 0u;
 542   3      
 543   3                      /* Dummy NAK to release bus */
 544   3                      EZI2C_1_CSR_REG = EZI2C_1_CSR_NAK;
 545   3                      break;
 546   3      
 547   3              }  /* End switch/case EZI2C_1_curState */
 548   2      
 549   2          }  
C51 COMPILER V9.51   EZI2C_1_INT                                                           01/04/2014 15:52:40 PAGE 10  

 550   1          else
 551   1          {
 552   2              /* Intentional blank line */       
 553   2          } 
 554   1      
 555   1          /* Check if Stop was detected */
 556   1          if(EZI2C_1_IS_BIT_SET(EZI2C_1_CSR_REG, EZI2C_1_CSR_STOP_STATUS))
 557   1          {
 558   2              /* Clear Busy Flag */
 559   2              EZI2C_1_curStatus &= ((uint8) ~EZI2C_1_STATUS_BUSY);
 560   2      
 561   2              /* error or stop - reset state */
 562   2              EZI2C_1_curState = EZI2C_1_SM_IDLE;
 563   2      
 564   2              /* Disable interrupt on Stop */
 565   2              EZI2C_1_CFG_REG &= ((uint8) ~EZI2C_1_CFG_STOP_IE);
 566   2          }
 567   1      }
 568          
 569          #if(EZI2C_1_WAKEUP_ENABLED)
                  /*******************************************************************************
                  * Function Name: EZI2C_1_WAKEUP_ISR
                  ********************************************************************************
                  *
                  * Summary:
                  *  Empty interrupt handler to trigger after wakeup.
                  *
                  * Parameters:
                  *  void
                  *
                  * Return:
                  *  void
                  *
                  *******************************************************************************/
                  CY_ISR(EZI2C_1_WAKEUP_ISR)
                  {
                      EZI2C_1_wakeupSource = 1u;  /* I2C was wakeup source */
                      
                      /* The SCL is stretched until EZI2C_SlaveSetWakeMode() is called */
                  }
              #endif /* (EZI2C_1_WAKEUP_ENABLED) */
 591          
 592          /* [] END OF FILE */
C51 COMPILER V9.51   EZI2C_1_INT                                                           01/04/2014 15:52:40 PAGE 11  

ASSEMBLY LISTING OF GENERATED OBJECT CODE


             ; FUNCTION EZI2C_1_ISR (BEGIN)
0000 C0E0              PUSH    ACC
0002 C083              PUSH    DPH
0004 C082              PUSH    DPL
0006 C085              PUSH    DPH1
0008 C084              PUSH    DPL1
000A C086              PUSH    DPS
000C 758600            MOV     DPS,#00H
000F C000        E     PUSH    ?C?XPAGE1SFR
0011 750000      E     MOV     ?C?XPAGE1SFR,#?C?XPAGE1RST
0014 C0D0              PUSH    PSW
0016 75D000            MOV     PSW,#00H
0019 C000              PUSH    AR0
001B C001              PUSH    AR1
001D C002              PUSH    AR2
001F C003              PUSH    AR3
0021 C004              PUSH    AR4
0023 C005              PUSH    AR5
0025 C006              PUSH    AR6
0027 C007              PUSH    AR7
                                           ; SOURCE LINE # 86
                                           ; SOURCE LINE # 105
0029 9049D7            MOV     DPTR,#049D7H
002C E0                MOVX    A,@DPTR
002D FF                MOV     R7,A
002E 900000      R     MOV     DPTR,#tmpCsr
0031 EF                MOV     A,R7
0032 F0                MOVX    @DPTR,A
                                           ; SOURCE LINE # 110
0033 900000      R     MOV     DPTR,#tmpCsr
0036 E0                MOVX    A,@DPTR
0037 FF                MOV     R7,A
0038 EF                MOV     A,R7
0039 5408              ANL     A,#08H
003B FF                MOV     R7,A
003C 7E00              MOV     R6,#00H
003E EF                MOV     A,R7
003F 6408              XRL     A,#08H
0041 4E                ORL     A,R6
0042 7004              JNZ     ?C0002
0044 7F01              MOV     R7,#01H
0046 8002              SJMP    ?C0003
0048         ?C0002:
0048 7F00              MOV     R7,#00H
004A         ?C0003:
004A EF                MOV     A,R7
004B 7003              JNZ     $ + 5H
004D 020000      R     LJMP    ?C0001
                                           ; SOURCE LINE # 111
                                           ; SOURCE LINE # 203
0050 9049D8            MOV     DPTR,#049D8H
0053 E0                MOVX    A,@DPTR
0054 FF                MOV     R7,A
0055 EF                MOV     A,R7
0056 5401              ANL     A,#01H
0058 FF                MOV     R7,A
0059 7E00              MOV     R6,#00H
005B EF                MOV     A,R7
005C 6401              XRL     A,#01H
C51 COMPILER V9.51   EZI2C_1_INT                                                           01/04/2014 15:52:40 PAGE 12  

005E 4E                ORL     A,R6
005F 7004              JNZ     ?C0005
0061 7F01              MOV     R7,#01H
0063 8002              SJMP    ?C0006
0065         ?C0005:
0065 7F00              MOV     R7,#00H
0067         ?C0006:
0067 EF                MOV     A,R7
0068 6047              JZ      ?C0004
                                           ; SOURCE LINE # 204
                                           ; SOURCE LINE # 207
006A 900000      E     MOV     DPTR,#EZI2C_1_dataPtrS1
006D 120000      E     LCALL   ?C?PLDXDATA
0070 900000      E     MOV     DPTR,#EZI2C_1_rwOffsetS1
0073 E0                MOVX    A,@DPTR
0074 FF                MOV     R7,A
0075 E9                MOV     A,R1
0076 2F                ADD     A,R7
0077 F9                MOV     R1,A
0078 E4                CLR     A
0079 3A                ADDC    A,R2
007A FA                MOV     R2,A
007B 120000      E     LCALL   ?C?CLDPTR
007E FF                MOV     R7,A
007F 9049D8            MOV     DPTR,#049D8H
0082 EF                MOV     A,R7
0083 F0                MOVX    @DPTR,A
                                           ; SOURCE LINE # 210
0084 9049D7            MOV     DPTR,#049D7H
0087 7414              MOV     A,#014H
0089 F0                MOVX    @DPTR,A
                                           ; SOURCE LINE # 213
008A 900000      E     MOV     DPTR,#EZI2C_1_rwOffsetS1
008D E0                MOVX    A,@DPTR
008E FF                MOV     R7,A
008F 900000      E     MOV     DPTR,#EZI2C_1_rwIndexS1
0092 EF                MOV     A,R7
0093 F0                MOVX    @DPTR,A
                                           ; SOURCE LINE # 216
0094 900000      E     MOV     DPTR,#EZI2C_1_rwIndexS1
0097 E0                MOVX    A,@DPTR
0098 04                INC     A
0099 F0                MOVX    @DPTR,A
                                           ; SOURCE LINE # 219
009A 900000      E     MOV     DPTR,#EZI2C_1_curStatus
009D E0                MOVX    A,@DPTR
009E FF                MOV     R7,A
009F EF                MOV     A,R7
00A0 4411              ORL     A,#011H
00A2 FF                MOV     R7,A
00A3 900000      E     MOV     DPTR,#EZI2C_1_curStatus
00A6 EF                MOV     A,R7
00A7 F0                MOVX    @DPTR,A
                                           ; SOURCE LINE # 222
00A8 900000      E     MOV     DPTR,#EZI2C_1_curState
00AB 7408              MOV     A,#08H
00AD F0                MOVX    @DPTR,A
                                           ; SOURCE LINE # 223
00AE 020000      R     LJMP    ?C0008
00B1         ?C0004:
                                           ; SOURCE LINE # 225
                                           ; SOURCE LINE # 228
C51 COMPILER V9.51   EZI2C_1_INT                                                           01/04/2014 15:52:40 PAGE 13  

00B1 9049D7            MOV     DPTR,#049D7H
00B4 7410              MOV     A,#010H
00B6 F0                MOVX    @DPTR,A
                                           ; SOURCE LINE # 231
00B7 900000      E     MOV     DPTR,#EZI2C_1_curStatus
00BA E0                MOVX    A,@DPTR
00BB FF                MOV     R7,A
00BC EF                MOV     A,R7
00BD 4412              ORL     A,#012H
00BF FF                MOV     R7,A
00C0 900000      E     MOV     DPTR,#EZI2C_1_curStatus
00C3 EF                MOV     A,R7
00C4 F0                MOVX    @DPTR,A
                                           ; SOURCE LINE # 234
00C5 900000      E     MOV     DPTR,#EZI2C_1_curState
00C8 7401              MOV     A,#01H
00CA F0                MOVX    @DPTR,A
                                           ; SOURCE LINE # 237
00CB 9049D6            MOV     DPTR,#049D6H
00CE E0                MOVX    A,@DPTR
00CF FF                MOV     R7,A
00D0 EF                MOV     A,R7
00D1 4410              ORL     A,#010H
00D3 FF                MOV     R7,A
00D4 EF                MOV     A,R7
00D5 F0                MOVX    @DPTR,A
                                           ; SOURCE LINE # 238
                                           ; SOURCE LINE # 240
00D6 020000      R     LJMP    ?C0008
00D9         ?C0001:
                                           ; SOURCE LINE # 241
00D9 900000      R     MOV     DPTR,#tmpCsr
00DC E0                MOVX    A,@DPTR
00DD FF                MOV     R7,A
00DE EF                MOV     A,R7
00DF 5401              ANL     A,#01H
00E1 FF                MOV     R7,A
00E2 7E00              MOV     R6,#00H
00E4 EF                MOV     A,R7
00E5 6401              XRL     A,#01H
00E7 4E                ORL     A,R6
00E8 7004              JNZ     ?C0010
00EA 7F01              MOV     R7,#01H
00EC 8002              SJMP    ?C0011
00EE         ?C0010:
00EE 7F00              MOV     R7,#00H
00F0         ?C0011:
00F0 EF                MOV     A,R7
00F1 7003              JNZ     $ + 5H
00F3 020000      R     LJMP    ?C0008
                                           ; SOURCE LINE # 242
                                           ; SOURCE LINE # 245
00F6 900000      E     MOV     DPTR,#EZI2C_1_curState
00F9 E0                MOVX    A,@DPTR
00FA FF                MOV     R7,A
00FB EF                MOV     A,R7
00FC 120000      E     LCALL   ?C?CCASE
00FF 0000        R     DW      ?C0013
0101 01                DB      01H
0102 0000        R     DW      ?C0016
0104 04                DB      04H
0105 0000        R     DW      ?C0019
C51 COMPILER V9.51   EZI2C_1_INT                                                           01/04/2014 15:52:40 PAGE 14  

0107 08                DB      08H
0108 0000              DW      00H
010A 0000        R     DW      ?C0024
                                           ; SOURCE LINE # 246
                                           ; SOURCE LINE # 248
010C         ?C0013:
                                           ; SOURCE LINE # 253
010C 9049D8            MOV     DPTR,#049D8H
010F E0                MOVX    A,@DPTR
0110 FF                MOV     R7,A
0111 900000      R     MOV     DPTR,#tmp8
0114 EF                MOV     A,R7
0115 F0                MOVX    @DPTR,A
                                           ; SOURCE LINE # 254
0116 900000      R     MOV     DPTR,#tmp8
0119 E0                MOVX    A,@DPTR
011A FF                MOV     R7,A
011B 7E00              MOV     R6,#00H
011D 900000      E     MOV     DPTR,#EZI2C_1_bufSizeS1
0120 E0                MOVX    A,@DPTR
0121 FC                MOV     R4,A
0122 A3                INC     DPTR
0123 E0                MOVX    A,@DPTR
0124 FD                MOV     R5,A
0125 C3                CLR     C
0126 EF                MOV     A,R7
0127 9D                SUBB    A,R5
0128 EE                MOV     A,R6
0129 9C                SUBB    A,R4
012A 5023              JNC     ?C0014
                                           ; SOURCE LINE # 255
                                           ; SOURCE LINE # 257
012C 9049D7            MOV     DPTR,#049D7H
012F 7410              MOV     A,#010H
0131 F0                MOVX    @DPTR,A
                                           ; SOURCE LINE # 260
0132 900000      R     MOV     DPTR,#tmp8
0135 E0                MOVX    A,@DPTR
0136 FF                MOV     R7,A
0137 900000      E     MOV     DPTR,#EZI2C_1_rwOffsetS1
013A EF                MOV     A,R7
013B F0                MOVX    @DPTR,A
                                           ; SOURCE LINE # 263
013C 900000      R     MOV     DPTR,#tmp8
013F E0                MOVX    A,@DPTR
0140 FF                MOV     R7,A
0141 900000      E     MOV     DPTR,#EZI2C_1_rwIndexS1
0144 EF                MOV     A,R7
0145 F0                MOVX    @DPTR,A
                                           ; SOURCE LINE # 266
0146 900000      E     MOV     DPTR,#EZI2C_1_curState
0149 7404              MOV     A,#04H
014B F0                MOVX    @DPTR,A
                                           ; SOURCE LINE # 267
014C 020000      R     LJMP    ?C0008
014F         ?C0014:
                                           ; SOURCE LINE # 269
                                           ; SOURCE LINE # 271
014F 9049D7            MOV     DPTR,#049D7H
0152 E4                CLR     A
0153 F0                MOVX    @DPTR,A
                                           ; SOURCE LINE # 272
C51 COMPILER V9.51   EZI2C_1_INT                                                           01/04/2014 15:52:40 PAGE 15  

                                           ; SOURCE LINE # 287
0154 020000      R     LJMP    ?C0008
                                           ; SOURCE LINE # 323
0157         ?C0016:
                                           ; SOURCE LINE # 326
0157 900000      E     MOV     DPTR,#EZI2C_1_rwIndexS1
015A E0                MOVX    A,@DPTR
015B FF                MOV     R7,A
015C 7E00              MOV     R6,#00H
015E 900000      E     MOV     DPTR,#EZI2C_1_wrProtectS1
0161 E0                MOVX    A,@DPTR
0162 FC                MOV     R4,A
0163 A3                INC     DPTR
0164 E0                MOVX    A,@DPTR
0165 FD                MOV     R5,A
0166 C3                CLR     C
0167 EF                MOV     A,R7
0168 9D                SUBB    A,R5
0169 EE                MOV     A,R6
016A 9C                SUBB    A,R4
016B 5033              JNC     ?C0017
                                           ; SOURCE LINE # 327
                                           ; SOURCE LINE # 329
016D 9049D8            MOV     DPTR,#049D8H
0170 E0                MOVX    A,@DPTR
0171 FF                MOV     R7,A
0172 900000      R     MOV     DPTR,#tmp8
0175 EF                MOV     A,R7
0176 F0                MOVX    @DPTR,A
                                           ; SOURCE LINE # 332
0177 9049D7            MOV     DPTR,#049D7H
017A 7410              MOV     A,#010H
017C F0                MOVX    @DPTR,A
                                           ; SOURCE LINE # 335
017D 900000      R     MOV     DPTR,#tmp8
0180 E0                MOVX    A,@DPTR
0181 FF                MOV     R7,A
0182 900000      E     MOV     DPTR,#EZI2C_1_dataPtrS1
0185 120000      E     LCALL   ?C?PLDXDATA
0188 900000      E     MOV     DPTR,#EZI2C_1_rwIndexS1
018B E0                MOVX    A,@DPTR
018C FE                MOV     R6,A
018D E9                MOV     A,R1
018E 2E                ADD     A,R6
018F F9                MOV     R1,A
0190 E4                CLR     A
0191 3A                ADDC    A,R2
0192 FA                MOV     R2,A
0193 EF                MOV     A,R7
0194 120000      E     LCALL   ?C?CSTPTR
                                           ; SOURCE LINE # 338
0197 900000      E     MOV     DPTR,#EZI2C_1_rwIndexS1
019A E0                MOVX    A,@DPTR
019B 04                INC     A
019C F0                MOVX    @DPTR,A
                                           ; SOURCE LINE # 339
019D 020000      R     LJMP    ?C0008
01A0         ?C0017:
                                           ; SOURCE LINE # 341
                                           ; SOURCE LINE # 343
01A0 9049D7            MOV     DPTR,#049D7H
01A3 E4                CLR     A
C51 COMPILER V9.51   EZI2C_1_INT                                                           01/04/2014 15:52:40 PAGE 16  

01A4 F0                MOVX    @DPTR,A
                                           ; SOURCE LINE # 344
                                           ; SOURCE LINE # 345
01A5 020000      R     LJMP    ?C0008
                                           ; SOURCE LINE # 349
01A8         ?C0019:
                                           ; SOURCE LINE # 352
01A8 900000      R     MOV     DPTR,#tmpCsr
01AB E0                MOVX    A,@DPTR
01AC FF                MOV     R7,A
01AD EF                MOV     A,R7
01AE 5402              ANL     A,#02H
01B0 FF                MOV     R7,A
01B1 7E00              MOV     R6,#00H
01B3 EF                MOV     A,R7
01B4 4E                ORL     A,R6
01B5 704C              JNZ     ?C0020
                                           ; SOURCE LINE # 353
                                           ; SOURCE LINE # 355
01B7 900000      E     MOV     DPTR,#EZI2C_1_rwIndexS1
01BA E0                MOVX    A,@DPTR
01BB FF                MOV     R7,A
01BC 7E00              MOV     R6,#00H
01BE 900000      E     MOV     DPTR,#EZI2C_1_bufSizeS1
01C1 E0                MOVX    A,@DPTR
01C2 FC                MOV     R4,A
01C3 A3                INC     DPTR
01C4 E0                MOVX    A,@DPTR
01C5 FD                MOV     R5,A
01C6 C3                CLR     C
01C7 EF                MOV     A,R7
01C8 9D                SUBB    A,R5
01C9 EE                MOV     A,R6
01CA 9C                SUBB    A,R4
01CB 5028              JNC     ?C0021
                                           ; SOURCE LINE # 356
                                           ; SOURCE LINE # 358
01CD 900000      E     MOV     DPTR,#EZI2C_1_dataPtrS1
01D0 120000      E     LCALL   ?C?PLDXDATA
01D3 900000      E     MOV     DPTR,#EZI2C_1_rwIndexS1
01D6 E0                MOVX    A,@DPTR
01D7 FF                MOV     R7,A
01D8 E9                MOV     A,R1
01D9 2F                ADD     A,R7
01DA F9                MOV     R1,A
01DB E4                CLR     A
01DC 3A                ADDC    A,R2
01DD FA                MOV     R2,A
01DE 120000      E     LCALL   ?C?CLDPTR
01E1 FF                MOV     R7,A
01E2 9049D8            MOV     DPTR,#049D8H
01E5 EF                MOV     A,R7
01E6 F0                MOVX    @DPTR,A
                                           ; SOURCE LINE # 361
01E7 9049D7            MOV     DPTR,#049D7H
01EA 7404              MOV     A,#04H
01EC F0                MOVX    @DPTR,A
                                           ; SOURCE LINE # 364
01ED 900000      E     MOV     DPTR,#EZI2C_1_rwIndexS1
01F0 E0                MOVX    A,@DPTR
01F1 04                INC     A
01F2 F0                MOVX    @DPTR,A
C51 COMPILER V9.51   EZI2C_1_INT                                                           01/04/2014 15:52:40 PAGE 17  

                                           ; SOURCE LINE # 365
01F3 8042              SJMP    ?C0008
01F5         ?C0021:
                                           ; SOURCE LINE # 367
                                           ; SOURCE LINE # 369
01F5 9049D8            MOV     DPTR,#049D8H
01F8 74FF              MOV     A,#0FFH
01FA F0                MOVX    @DPTR,A
                                           ; SOURCE LINE # 372
01FB 9049D7            MOV     DPTR,#049D7H
01FE 7404              MOV     A,#04H
0200 F0                MOVX    @DPTR,A
                                           ; SOURCE LINE # 373
                                           ; SOURCE LINE # 374
0201 8034              SJMP    ?C0008
0203         ?C0020:
                                           ; SOURCE LINE # 376
                                           ; SOURCE LINE # 378
0203 9049D8            MOV     DPTR,#049D8H
0206 74FF              MOV     A,#0FFH
0208 F0                MOVX    @DPTR,A
                                           ; SOURCE LINE # 381
0209 9049D7            MOV     DPTR,#049D7H
020C E4                CLR     A
020D F0                MOVX    @DPTR,A
                                           ; SOURCE LINE # 384
020E 900000      E     MOV     DPTR,#EZI2C_1_curStatus
0211 E0                MOVX    A,@DPTR
0212 FF                MOV     R7,A
0213 EF                MOV     A,R7
0214 54EF              ANL     A,#0EFH
0216 FF                MOV     R7,A
0217 900000      E     MOV     DPTR,#EZI2C_1_curStatus
021A EF                MOV     A,R7
021B F0                MOVX    @DPTR,A
                                           ; SOURCE LINE # 387
021C 900000      E     MOV     DPTR,#EZI2C_1_curState
021F E4                CLR     A
0220 F0                MOVX    @DPTR,A
                                           ; SOURCE LINE # 389
                                           ; SOURCE LINE # 390
0221 8014              SJMP    ?C0008
                                           ; SOURCE LINE # 533
0223         ?C0024:
                                           ; SOURCE LINE # 535
0223 900000      E     MOV     DPTR,#EZI2C_1_curState
0226 E4                CLR     A
0227 F0                MOVX    @DPTR,A
                                           ; SOURCE LINE # 538
0228 900000      E     MOV     DPTR,#EZI2C_1_rwOffsetS1
022B E4                CLR     A
022C F0                MOVX    @DPTR,A
                                           ; SOURCE LINE # 541
022D 900000      E     MOV     DPTR,#EZI2C_1_rwIndexS1
0230 E4                CLR     A
0231 F0                MOVX    @DPTR,A
                                           ; SOURCE LINE # 544
0232 9049D7            MOV     DPTR,#049D7H
0235 E4                CLR     A
0236 F0                MOVX    @DPTR,A
                                           ; SOURCE LINE # 545
                                           ; SOURCE LINE # 547
C51 COMPILER V9.51   EZI2C_1_INT                                                           01/04/2014 15:52:40 PAGE 18  

                                           ; SOURCE LINE # 549
                                           ; SOURCE LINE # 551
                                           ; SOURCE LINE # 553
0237         ?C0008:
                                           ; SOURCE LINE # 556
0237 9049D7            MOV     DPTR,#049D7H
023A E0                MOVX    A,@DPTR
023B FF                MOV     R7,A
023C EF                MOV     A,R7
023D 5420              ANL     A,#020H
023F FF                MOV     R7,A
0240 7E00              MOV     R6,#00H
0242 EF                MOV     A,R7
0243 6420              XRL     A,#020H
0245 4E                ORL     A,R6
0246 7004              JNZ     ?C0027
0248 7F01              MOV     R7,#01H
024A 8002              SJMP    ?C0028
024C         ?C0027:
024C 7F00              MOV     R7,#00H
024E         ?C0028:
024E EF                MOV     A,R7
024F 601E              JZ      ?C0029
                                           ; SOURCE LINE # 557
                                           ; SOURCE LINE # 559
0251 900000      E     MOV     DPTR,#EZI2C_1_curStatus
0254 E0                MOVX    A,@DPTR
0255 FF                MOV     R7,A
0256 EF                MOV     A,R7
0257 54EF              ANL     A,#0EFH
0259 FF                MOV     R7,A
025A 900000      E     MOV     DPTR,#EZI2C_1_curStatus
025D EF                MOV     A,R7
025E F0                MOVX    @DPTR,A
                                           ; SOURCE LINE # 562
025F 900000      E     MOV     DPTR,#EZI2C_1_curState
0262 E4                CLR     A
0263 F0                MOVX    @DPTR,A
                                           ; SOURCE LINE # 565
0264 9049D6            MOV     DPTR,#049D6H
0267 E0                MOVX    A,@DPTR
0268 FF                MOV     R7,A
0269 EF                MOV     A,R7
026A 54EF              ANL     A,#0EFH
026C FF                MOV     R7,A
026D EF                MOV     A,R7
026E F0                MOVX    @DPTR,A
                                           ; SOURCE LINE # 566
                                           ; SOURCE LINE # 567
026F         ?C0029:
026F D007              POP     AR7
0271 D006              POP     AR6
0273 D005              POP     AR5
0275 D004              POP     AR4
0277 D003              POP     AR3
0279 D002              POP     AR2
027B D001              POP     AR1
027D D000              POP     AR0
027F D0D0              POP     PSW
0281 D000        E     POP     ?C?XPAGE1SFR
0283 D086              POP     DPS
0285 D084              POP     DPL1
C51 COMPILER V9.51   EZI2C_1_INT                                                           01/04/2014 15:52:40 PAGE 19  

0287 D085              POP     DPH1
0289 D082              POP     DPL
028B D083              POP     DPH
028D D0E0              POP     ACC
028F 32                RETI    
             ; FUNCTION EZI2C_1_ISR (END)



MODULE INFORMATION:   STATIC OVERLAYABLE
   CODE SIZE        =    656    ----
   CONSTANT SIZE    =   ----    ----
   XDATA SIZE       =      2    ----
   PDATA SIZE       =   ----    ----
   DATA SIZE        =   ----    ----
   IDATA SIZE       =   ----    ----
   BIT SIZE         =   ----    ----
   EDATA SIZE       =   ----    ----
   HDATA SIZE       =   ----    ----
   XDATA CONST SIZE =   ----    ----
   FAR CONST SIZE   =   ----    ----
END OF MODULE INFORMATION.


C51 COMPILATION COMPLETE.  0 WARNING(S),  0 ERROR(S)
